:020000040000FA
:1000000080312528013401347E1480310B1F2328D0
:100010004E011E1B141F10288B31342380312328DE
:100020001B1A111E17288A31C8228031232817185D
:100030000D1C1E288D31BD258031232897188D1C5D
:1000400023288B31B9237E100900803127288A317B
:100050006E228031F900803102208031EC00803145
:1000600003208031ED00903084008B308500D73044
:100070008600003087000030FF0014308A31E02213
:10008000803170308400233085008030FE000030E5
:10009000FF008A31D4228031F601F701F801603087
:1000A0008400003085000C30FE000030FF008A31F3
:1000B000D4228031A0308400003085003730FE002B
:1000C0000030FF008A31D4227E1040018031682840
:1000D0004001DD01DC010030D8000030D9000030E3
:1000E000DA00DE018A31712280318A318722803143
:1000F00058018C1F7E28C4308E0084288A31AF229C
:1001000080318D31162580318B170B174001E601A8
:1001100099158A318722803140016608031DAC2978
:100120003C308A317D228031972890199A284E01DF
:10013000141F9528141FA42914138A31AF2280316B
:10014000D0304001D6005608A500B73085313025A3
:100150008031173040016206031DB82841013B0879
:100160003C04031DB82801304001D6005608EC00BD
:1001700041013B084001D6005608E200B730860036
:100180000030870020308400003085001230D60017
:1001900016001A00D60BC828843141248031400152
:1001A000D7005708DF005F080319EF286C08031910
:1001B000EF285F08D600D70156084101BB00400177
:1001C00057084101BC0040015F08D60056084101B4
:1001D000D200B7308B31FE2380314001EC0164083E
:1001E000743E840090300318013E85000008FF3EF5
:1001F000D600FF3003180030D7005708803A803C03
:10020000031D042956085C0203180C290130400123
:10021000D6005608DC0716294001DC010130D60063
:100220005608E407043064020318E401B73086007E
:10023000003087002C308400003085001230D6005A
:1002400016001A00D60B20296435E33E860087018C
:10025000413F8A00403F0A00813140012D08E10002
:100260002C08E0004101240840016106031D3C29DF
:10027000410123084001600603194A29A001A00A90
:10028000A101A10A6108A3006008A20001308D311C
:1002900082258031400161084101A40040016008CD
:1002A0004101A3004001DB01DB0A8A318722803152
:1002B000410152084001D6005608E90041015108A9
:1002C0004001D6005608EA00410150084001D6001E
:1002D0005608EB006D08031990296508031D902945
:1002E0000A305D02031882298B31A42380316930E2
:1002F0008631A02680314001DB010130D60056084E
:10030000DD079A29DD01ED010130D6005608E50030
:1003100058308631A02680318B31582380319A297C
:1003200058308631A02680314001650803199A298A
:10033000E501ED0140015B08D6005608A200640803
:100340008F3182278031AC29901DAC29901101306A
:100350004001D6005608E60040016603031D8C28C4
:100360008A31AF2280318B31A4238031C9304001E2
:10037000D6005608A500A5308531302580314001D2
:10038000A001A00AA101A10A0030A200A30001302F
:100390008D318225803104304001D6005608E300BB
:1003A0000230D6005608A20003308F3182278031F8
:1003B0004001E90141014F084001D6005608EA001A
:1003C000EB0169308631A026803140010E1A8F1D65
:1003D000E52905308A317D2280318A31A72280319A
:1003E0004E011E174E01911BFF2A901D932A0430C7
:1003F00040016306031D1D2A8F19092A6308D600D0
:100400005608D000A5308331212380314001DE0120
:10041000DE0AE9014101300885002F0884003030F0
:1004200084078830853D00084001D6005608EA0060
:10043000EB0169308631A02680310230400163062D
:10044000031D542A0E1A262A0330292A8F19332A0B
:100450000230D6005608D000A530833121238031E8
:100460004001DE01DE0A41012E0885002D088400CE
:10047000003084079030853D00084001D6005608C2
:10048000E90041012C0885002B0884000030840716
:100490009030853D00084001D6005608EA00EB0187
:1004A00069308631A026803140016303031D8F2A05
:1004B0000E1A612AD001D00AA53083312123803160
:1004C0006B2A8F196E2AD001A53083312123803108
:1004D0004101A501A6014001DE01DE0A41012A0811
:1004E000850029088400003084079030853D00088D
:1004F0004001D6005608E900410128088500270878
:100500008400003084079030853D00084001D6000B
:100510005608EA00EB0169308631A026803140019F
:10052000E8014E01901140016708031DE42AF229F9
:100530000230D6005608E30041012E0885002D0840
:100540008400003084079030853D00084001D600CB
:100550005608E90041012C0885002B088400003072
:1005600084079030853D00084001D6005608EA0017
:10057000EB0169308631A0268031EF2AE301E30ADE
:1005800041012A0885002908840000308407903042
:10059000853D00084001D6005608E90041012808C1
:1005A000850027088400003084079030853D0008CE
:1005B0004001D6005608EA00EB0169308631A026DA
:1005C0008031EF2AE301EF2A6308013A0319E22A96
:1005D000033A0319BE2A063A0319982AEF2A400162
:1005E00063080319FF2A0230D6005608A2006308E8
:1005F0008F31822780314001E701E801F2298A31F9
:10060000992280314001A20100308F318227803150
:1006100040015E080319102BA53087313227803145
:100620004001DE014E011E138B3158238031013011
:100630004001D6005608ED00DD01E801E701E601C2
:1006400089284001D50004305006031D4E2B550863
:100650000A3E86008701403FD100413FD200520848
:10066000803AD30088305302031D382B1F305102CB
:100670000318452B400155080A3E860087010130CA
:10068000810741310318810A4E2B400155080A3E6B
:1006900086008701D030C03F0730C13F033050068D
:1006A000031D792B5508083E86008701403FD10085
:1006B000413FD2005208803AD30080305302031DDC
:1006C000632B0C3051020318702B40015508083E73
:1006D000860087010130810741310318810A792B97
:1006E00040015508083E860087010130C03F0030B8
:1006F000C13F02305006031DCE2B5508083E860030
:100700008701403FD100413FD2006730510784004C
:100710009030523D85000008D3005308D4001C30AF
:100720005406031DA62B55080A3E86008701403F4C
:10073000F400413FF5008B3115238331003A031952
:10074000A62B1D304001D1005108D40040015508AE
:10075000063E86008701403FD100413FD20052084B
:10076000803AD30080305302031DB82B5408510245
:100770000318C52B40015508063E8600870101304D
:10078000810741310318810ACE2B40015508063EEE
:10079000860087010130C03F0030C13F5003031D78
:1007A000F72B5508043E86008701403FD100413FAA
:1007B000D2005208803AD30080305302031DE22B4E
:1007C000173051020318EF2B40015508043E8600F4
:1007D00087010130810741310318810AF72B40015D
:1007E0005508043E860087010030C03FC13F5008D5
:1007F000031D262C5508023E86008701403FD1008C
:10080000413FD2005208803AD30080305302031D8A
:100810000B2C3B3051020318182C40015508023EA6
:10082000860087010130810741310318810A202C9D
:1008300040015508023E860087010030C03FC13F9D
:100840005508860087010030C03FC13F550886002B
:1008500087012C308400003085001230D100160052
:100860001A00D10B2F2C8F3117274001D200D30152
:1008700055080C3E860087015208C03F5308C13F0F
:100880000800033040012806290403194C2C0A30C3
:1008900028062904031D2E2D2B08803AF4008730EA
:1008A0007402031D552CEA302A0203182E2DE23063
:1008B00040012A06073003192B06031D122D0A30AA
:1008C00028062904031D122D1C3026062704031DAB
:1008D000122D033024062504031D122D22082304A3
:1008E0000319102D122D033028062904031D882C0E
:1008F0001F3026062704031D882C023024062504F9
:10090000031D882C22082304031D882C03300800B3
:100910000A3028062904031D192D1B30260627043A
:10092000031D192D033024062504031D192D22084B
:1009300023040319102D192D033028062904031D43
:10094000AF2C1D3026062704031DAF2C02302406D1
:100950002504031DAF2C220823040319862C0A301A
:1009600028062904031D202D193026062704031DFF
:10097000202D033024062504031D202D22082304E6
:100980000319102D202D033028062904031DD62C11
:100990001C3026062704031DD62C0230240625040D
:1009A000031DD62C220823040319862C0A3028069E
:1009B0002904031D272D1F3026062704031D272D7C
:1009C000033024062504031D272D220823040319C0
:1009D000102D272D033028062904031DFD2C1B3064
:1009E00026062704031DFD2C023024062504031DC2
:1009F000FD2C220823040319862C0A30280629041A
:100A0000031D2E2D1E3026062704031D2E2D033018
:100A100024062504031D2E2D22082304031D2E2D3C
:100A200002300800E3302A06073003192B060319A9
:100A3000732CE4302A06073003192B0603199C2C6B
:100A4000E5302A06073003192B060319C32CE630BC
:100A50002A06073003192B060319EA2C0030080078
:100A60004001A80058010C1A08008C1610088C319F
:100A700036248531D03E4001A600073003180830E7
:100A8000A70028080A3E860087012608C03F2708DD
:100A9000C13F580110084001A6002508063E860007
:100AA000870126088100580111088C3136248531D0
:100AB0004001A600A7012808083E860087012608F5
:100AC000C03F2708C13F580111084001A600250872
:100AD000053E8600870126088100580112088C31E6
:100AE000362485314001A600A70128080C3E860067
:100AF00087012608C03F2708C13F5801120840015E
:100B0000A6002508033E86008701260881005801BB
:100B100013088C31362485314001A600A70128082E
:100B2000063E860087012608C03F2708C13F5801BE
:100B300013084001A6002508043E86008701260808
:100B40008100580114088C31362485314001A600FB
:100B5000A7012808043E860087012608C03F270811
:100B6000C13F580114084001A6002508023E860036
:100B7000870126088100580115088C3136248531FB
:100B80004001A600A7012808023E8600870126082A
:100B9000C03F2708C13F580115084001A600250A9B
:100BA0008600870126088100580116088C313624FA
:100BB0004001A600A7012808860087012608C03F3B
:100BC0002708C13F580116084001A60025088600E5
:100BD00087012608810058018C1208004001CB01D2
:100BE000CC013508803ABE0080303E02031DFA2D4C
:100BF00001303402031C082E40013508803ABE0043
:100C000080303E02031D062E0D303402031C0C2ED4
:100C10004001AC01AD01080040013708F50036087D
:100C2000F4008B31152385314001BE003E08CA0017
:100C30004A08CD013408FF3EBE00FF30353DBF00FD
:100C40003F08803A803C031D272E3E084D020318C2
:100C50004C2E40014D08BE00BF01BE35BF0D5030C7
:100C60003E07840090303F3D8500003FC400013FB7
:100C7000C5004D03031D432E4A03031D432EB83008
:100C8000C4000230C5004408CB074508CC3D013004
:100C9000BE003E08CD071A2E40013208FF3EA000DC
:100CA000FF30333DA1001830A2000030A3008C318A
:100CB0001A24853140012008CB072108CC3D30089B
:100CC000CB073108CC3D22304C02233003194B02B4
:100CD0000318842E4B08A0004C08A100A201A30118
:100CE0000030A7000030A6000030A5000F30A4009F
:100CF0008C31B124853140012308C9002208C80085
:100D00002108C70020088B2E0030C9000130C80020
:100D1000FF30C700FF30C6004608BE004708BF00CE
:100D20004808C0004908C1000730C136C00CBF0CDC
:100D3000BE0C890B952E3F08AD003E08AC000800A4
:100D40004001A6002608023E8600870101080F39EF
:100D5000F4007408A5002608023E860087010108F9
:100D6000F4000430F436890BB22E74080739F5000C
:100D70007508A000260A8600870101080F39F400D3
:100D80000330F435FF3E031DC12E7435F5007508A0
:100D9000A100260A860087010108F4000430F43619
:100DA000890BCF2E74080739F5007508A2002608B4
:100DB0008600870101080F39F4000330F435FF3E47
:100DC000031DDE2E7435F5007508A3002608860085
:100DD00087010108F4000130F435FF3E031DEC2EBD
:100DE0007435C039F5007508A400251CF92E981536
:100DF000FA2E9811A51CFE2E1815FF2E1811251D70
:100E0000032F9814042F9810A51D082F1814092FCC
:100E10001810F030F40074089C052008F4007408E1
:100E20009C040F30F40074089B052108F40074083A
:100E30009B04F030F40074089B052208F400740849
:100E40009B040F30F400740899052308F40074081B
:100E500099043F30F40074089A052408F4007408DB
:100E60009A0408004001A00058018C168C13400120
:100E700020080A3E86008701403FF400413FF5000C
:100E80003030740784008830753D850000085801B3
:100E9000900040012008083E86008701403FF40092
:100EA000413FF5000030740784009030753D8500A7
:100EB000000858019100400120080C3E860087017F
:100EC000403FF400413FF50000307407840090304B
:100ED000753D850000085801920040012008063E3B
:100EE00086008701403FF400413FF5000030740761
:100EF00084009030753D8500000858019300400142
:100F00002008043E86008701403FF400413FF50081
:100F10000030740784009030753D8500000858014A
:100F2000940040012008023E86008701403FF40003
:100F3000413FF5000030740784009030753D850016
:100F40000008580195004001200886008701403FB5
:100F5000F400413FF5000030740784009030753D87
:100F600085000008580196008C178C1FB52F8C1235
:100F7000080040019C019B01980199019A0196018A
:100F800050309200930117309400083095007E0194
:100F9000D9010430CE00C301E401B8010830DA0001
:100FA000E501C401B9011030CF00E601BA01C50165
:100FB000D001DB01013097007D014508E039093897
:100FC000C5004608E0391438C60002307E0194009E
:100FD000133099007D013B08E0391438BB00143010
:100FE0007E0198007D013E08E0391B38BE000230CA
:100FF0007E0196000800F50075088A3182220800FB
:1014DA0008000134780808008C315D240800813046
:1014EA0052018C000800F4007408450193000800BA
:1014FA00F50075088A3178220800F400740845015D
:10150A008D000800403051018D000F1A08008A2A08
:10151A0075084101EE007408ED00080075084101E4
:10152A00EC007408EB0008007C01AE134F011B1697
:10153A004E0191130800403043018F002030900083
:10154A008D0108004F011B127C01AE172E164E01A9
:10155A009113080002305101930060308D000F1A78
:10156A000800B42A4F0196019701980199019A013E
:10157A009B010800F4004301901374088C000F1CAF
:10158A00C42A0C0808004E01111240019213981740
:10159A0000004001941542019117111408006400DB
:1015AA00800101310130FE020030FF3B7F087E04DA
:1015BA0003190034D52AFE0012001E000130FE0273
:1015CA000030FF3B7F087E0403190034E12A6030B3
:1015DA0051018D0040308F00083091000230930095
:1015EA00900192019401080080304601960007306C
:1015FA009500C030940044011E08CF3910389E006F
:10160A00080001304501900020308F009101073019
:10161A008D008C014E019010F03045018E000800BB
:10162A00033074054001A00000307505A1002008B0
:10163A002104031D222B0130080000300800073066
:10164A0045019600063095000C3097003C30930017
:10165A0092014E019011FF304501940008000430B8
:10166A004001680203183E2B0130F0007008E807B9
:10167A00432BE8010130F0007008E7004E01141313
:10168A0008007C01AF01B0010330B1000A30B2009A
:10169A000A30B3000130B4000430B500B601B70116
:1016AA002E16AE0108004F01161398129B108B31AB
:1016BA00CF238B318A3174228B318D314C25013005
:1016CA004001A0002008F900080002307C019B00BC
:1016DA0012309C0020309D0009309E0009309F0086
:1016EA000230A000A101A201A30180309A000800E3
:1016FA0005307C01A500A6010A30A7000330A80026
:10170A000A30A9000230AA00AB012030AC00AD01BA
:10171A008130A40008000034033402340534003454
:10172A000334053401340434063402340434FE34F8
:10173A000D344D340E34AD340E34EE3405344E01CE
:10174A00971017101B127C0190134201911352013A
:10175A008C014001941592179A1198134F0116178C
:10176A0098169B14F90108004E018D100130F00003
:10177A0070084001ED000130F0007008F6004101E8
:10178A006B086C04031908006C088A006B080A00CD
:10179A008B3108007C0191012030920009309300BE
:1017AA000A3094000A309500023096000230970001
:1017BA0098019901903090004E0111121B160800F1
:1017CA0075084001A1007408A000A136A00CA1363A
:1017DA00A00C200846019500740803394001A000B6
:1017EA000530A035FF3E031DF62B20354601940037
:1017FA0008004001A00058018C168C1340012008F3
:10180A00043E86008701403FF400413FF500003066
:10181A00740784009030753D8500000858019400D3
:10182A008C178C1F162C8C120800F401F50140014C
:10183A00201C232C2208F4072308F53D0130A23589
:10184A00A30D890B242C0130A136A00C890B292C5D
:10185A0020082104031D1C2C7508A1007408A0008F
:10186A0008004001A4002408F4000430F436890B6F
:10187A003B2C74080F39F5007508A00024080F39AD
:10188A00F4007408A100A201A3012008220203188F
:10189A00572C0A30F4007408A3070130F4007408C6
:1018AA00A2074A2C2108F4007408A3072308080099
:1018BA008A31B7228C318731B9278C318A31EC22AF
:1018CA008C318A31A0228C318A3174228C318D314B
:1018DA004C258C318B316A238C318B3124238C310A
:1018EA008B3106238C318B31CF238C318B314623BC
:1018FA008C318B317D238C318A31F92208004001E9
:10190A00270828040319AC2CAB01AB0AA81B972C97
:10191A000130A735A80D890B8E2C0130F50075080A
:10192A00AB078B2C28082A02031D9D2C27082902A5
:10193A00031CA32C2708A9022808AA3B0130A836B1
:10194A00A70C890BA42C0130AB02031D972C2A0883
:10195A00A8002908A700080000304001AB000030A9
:10196A00AA000030A9000030A800201CC42C2408BA
:10197A00A8072508A93D2608AA3D2708AB3D01303E
:10198A00A435A50DA60DA70D890BC52C0130A336CC
:10199A00A20CA10CA00C890BCC2C23082204210434
:1019AA002004031DBA2C2B08A3002A08A200290828
:1019BA00A1002808A00008004001A501A6012008EE
:1019CA0021040319112DA401A40AA11BF62C01302C
:1019DA00A035A10D890BED2C0130F4007408A40781
:1019EA00EA2C0130A535A60D890BF72C2108230214
:1019FA00031D012D20082202031C082D2008A20223
:101A0A002108A33B25140130A136A00C890B092D0E
:101A1A000130A402031DF62C2608A1002508A00007
:101A2A00080058018C168C138A316F228D31003AC6
:101A3A00031D302D183058019000103091000630E7
:101A4A00920006309300173094000230950053300C
:101A5A009600F801F80A58018E130A308F000530F3
:101A6A009700063098002630990015309A001730F2
:101A7A009B0053309C008E17C4308E0007308D00B7
:101A8A008C178C1F462D8C124E011413080041012D
:101A9A008C018D014A308E0001308F009201930132
:101AAA00980104309A0012309F00E83042018C00FD
:101ABA0003308D008E018F01900192012030930036
:101ACA0006309400950103309600970198019430EE
:101ADA0091004E010D1017146D30F4000A30F50014
:101AEA008A318D228D314E018D1097146D30F4009C
:101AFA000A30F5008A31932208004001A600A901A4
:101B0A00AA01FF30A2050330A3052608031D2A17E0
:101B1A002008031DAA162108031D2A162308A5005A
:101B2A002208A400A435A50DA435A50D2408A904EE
:101B3A002508AA042A08A4002408A7002908A40042
:101B4A002408A8004F011A128A31A0228D314001BF
:101B5A00191127088A31BF228D31400128088A319C
:101B6A00BF2240011915430190014F011A160800BE
:101B7A004E010D1040019A159411420111141118C9
:101B8A00C42D4E010D1040019A1194159217770831
:101B9A00F000F101F035F10D7030F2002330F3005E
:101BAA007008720786007108733D870041011008AA
:101BBA00C03F1108C13F0130F0007008F7073F30FD
:101BCA00F0007008F7054E018D1CF02D76080319F8
:101BDA00F12D8D10F12DF6014201911341016D088D
:101BEA006E04031908006E088A006D080A008D3118
:101BFA00080040013008A0003108A100890D893B86
:101C0A008909A200A3000030A7000030A600153001
:101C1A00A5005530A4008C31B1248D314001230830
:101C2A00C5002208C4002108C3002008C2002E08EB
:101C3A00A0002F08A100890D893B8909A200A300F1
:101C4A000030A7000030A6000030A5005B30A400D9
:101C5A008C31B1248D3140012008C2072108C33DCF
:101C6A002208C43D2308C53D4208BE004308BF0000
:101C7A004408C0004508C1000730C136C00CBF0C7B
:101C8A00BE0C890B422E3F08AD003E08AC0008008E
:101C9A00400138083904031D572E0630B8000030B9
:101CAA00B9005B2EFF30B807FF30B93D3908A100F3
:101CBA003808A000A030A2000530A3008C311A24F5
:101CCA008E3140012108C7002008C6003108A10052
:101CDA003008A0003C30A2000030A3008C311A2446
:101CEA008E3140012008C6072108C73D2E08C607C5
:101CFA002F08C73D4608A0004708A100A201A3017A
:101D0A000030A7000030A6000030A5000D30A40066
:101D1A008C31B1248E3140012308C5002208C40049
:101D2A002108C3002008C2004208BE004308BF00C1
:101D3A004408C0004508C1000730C136C00CBF0CBA
:101D4A00BE0C890BA22E3F08AD003E08AC0008006D
:101D5A0040013208FF3EA000FF30333DA100183099
:101D6A00A2000030A3008C311A248E3140012108D0
:101D7A00C3002008C2003008C2073108C33DDB2E69
:101D8A005830D72E3708F5003608F4008B31152362
:101D9A008E31003A0319D32E5E30D42E61304001C1
:101DAA00D72E5B30C0000030C100F92E35088500FF
:101DBA00340884008435850D4E3084079030853D83
:101DCA00003FBE00013FBF003F08023A0319EE2E52
:101DDA00F92E3E08A03A0319C72E703A0319D62ED7
:101DEA00383A0319C52EF92E4108A1004008A0006F
:101DFA004308A3004208A2008C311A248E31400104
:101E0A002108C3002008C2004308BF004208BE00E0
:101E1A000630BF36BE0C890B0E2F3E08AC003F08B9
:101E2A00AD00080040013708CF003608CE0035085B
:101E3A00CD003408CC003308CB003208CA00003089
:101E4A004D02033003194C0203182D2F01302E2F97
:101E5A000030BE00BF013E08CE023F08CF3B07302C
:101E6A00A7000030A8004C08D63E8600870101086A
:101E7A00BE00BF019030A0000130A1004F08A300AE
:101E8A004E08A2008C31E1248F3140014F08C10075
:101E9A004E08C000C136C00CC136C00C200840072D
:101EAA00C2002108413DC3003E084207C4003F0862
:101EBA00433DC5006430A0000030A1004F08A300D4
:101ECA004E08A2008C31E1248F31400120084402DF
:101EDA00C6002108453BC7004E084607C8004F0800
:101EEA00473DC9004A084807A9004B08493DAA00CE
:101EFA008C3184244001270808004001A300AB2F3D
:101F0A004601961345018E137C019A13400112175C
:101F1A00962F4601961745018E177C019A174001A4
:101F2A0012131216B92F4601961745018E177C0116
:101F3A009A1740011217A92F4601961745018E17C5
:101F4A007C019A17400112131212B92F2308003A82
:101F5A000319852F013A03198E2F033A0319982F73
:101F6A00013A0319A12FB92F51010E0E0739043A6C
:101F7A00031DC32F8F3045018E05F32F0E0E07392F
:101F8A00063A031DF32F703045018E04F32F0730F4
:101F9A008731FB278F311430F4000030F5008B3184
:101FAA00E5237C01A111080007308731FB278F3117
:101FBA000230F4000030F5008B31E5237C01A111D9
:101FCA00080007308731FB278F311430F4000030C6
:101FDA00F5008B31E5237C01A11508004001220898
:101FEA00003A0319CC2F013A0319D92F033A0319DE
:101FFA00E62FFF2F0800003401340234033404347E
:10200A0005340634073408340934103411341234D0
:10201A00133414341534163417341834193420345C
:10202A0021342234233424342534263427342834E2
:10203A002934303431343234333434343534363468
:10204A0037343834393440344134423443344434F4
:10205A004534463447344834493450345134523480
:10206A00533454345534563457345834593460340C
:10207A006134623463346434653466346734683492
:10208A006934703471347234733474347534763418
:10209A00773478347934E8340234A0340234E834BA
:1020AA000234D0340234E8340234D0340234E8340E
:1020BA000234E8340234D0340234E8340234D034FE
:1020CA000234E83402341F341C341F341E341F34E3
:1020DA001E341F341F341E341F341E341F34193467
:0620EA0005340534053445
:020000040001F9
:0A000E00E81DFF3D9F3FFF1FFF3F6D
:00000001FF
